:1000000066C180C17FC17EC17DC17CC1F0C27AC1A1
:1000100079C178C177C1F7C12DC274C173C172C1F2
:1000200071C170C16FC10A0D496E746572616374EC
:10003000697665204D6F64650A0D0A0D302E2E37E6
:100040002020202020526576657273652043686108
:100050006E6E656C20302E2E372028616E64207203
:10006000657365742074696D6572290A0D412E2EC1
:10007000482020202020536574204368616E6E65FF
:100080006C20302E2E37206F6E0A0D612E2E6820C8
:1000900020202020536574204368616E6E656C20BB
:1000A000302E2E37206F66660A0D455343202020E0
:1000B00020202052657475726E2066726F6D204923
:1000C0006E746572616374697665204D6F64650A4C
:1000D0000D0A0D3E2020000A0D436F6D6D616E64A8
:1000E000204D6F64650A0D0A0D20204D414E55418B
:1000F0004C202020202020202020202020202020D4
:1001000020202020202020202020202020202020EF
:10011000202020202020202D2D2053746172742057
:10012000496E746572616374697665204D6F6465AC
:100130000A0D2020434F4E464947204368616E6EAA
:10014000656C204F6E204F66662052616E646F6D45
:100150005F4F6E2052616E646F6D5F4F6666202048
:100160002D2D205365742054696D6520436F6E6694
:1001700069670A0D20205341564520202020202069
:10018000202020202020202020202020202020206F
:10019000202020202020202020202020202020205F
:1001A00020202D2D205361766520746F2045455009
:1001B000524F4D0A0D20204C49535420202020201E
:1001C000202020202020202020202020202020202F
:1001D000202020202020202020202020202020201F
:1001E0002020202D2D20446973706C617920437587
:1001F00072656E742053657474696E67730A0D00BE
:100200000A0D0A0D547261696E2054696D65720A97
:100210000D2D2D2D2D2D2D2D2D2D2D2D2D2D2D2D2E
:100220002D0A0D286329206D69686F203230313323
:10023000205757572E4D4C41422E435A0A0D312E0E
:1002400030300A0D0A0D00434F4D4D414E442020E1
:10025000204348414E4E454C2020202054494D45D6
:100260005F4F4E202054494D455F4F464620202089
:1002700020524E445F4F4E20202020524E445F4F6C
:1002800046460A0D2D2D2D2D2D2D2D2D2D2D2D2DAF
:100290002D2D2D2D2D2D2D2D2D2D2D2D2D2D2D2D8E
:1002A0002D2D2D2D2D2D2D2D2D2D2D2D2D2D2D2D7E
:1002B0002D2D2D2D2D2D2D2D2D2D2D2D2D2D2D0A91
:1002C0000D006364696E6F70737578585B0011245C
:1002D0001FBECFE5D4E0DEBFCDBF11E0A0E6B0E0A9
:1002E000E0EEFCE102C005900D92A833B107D9F70A
:1002F00012E0A8E3B1E001C01D92A53AB107E1F711
:100300000AD3ECCC7DCE9C01E199FECF3FBB2EBB46
:10031000E09A8DB308959C01E199FECF3FBB2EBBBF
:100320006DBB0FB6F894E29AE19A0FBE089588303B
:1003300028F5A82FB0E09D01220F331FF901EA52E2
:10034000FF4F0190F081E02D8081AA50BF4F9C911A
:10035000892B8083AC91F901EA51FF4F662339F074
:100360000190F081E02D80818A2B80830895019097
:10037000F081E02D8081A095A823A0830895CF93DC
:10038000DF93883010F040E01CC0282F30E0D90106
:10039000AA0FBB1FFD01E250FF4F0190F081E02D3D
:1003A0008081225E3E4FE9019881892B8083A25F84
:1003B000BE4FED91FC91808140E09881892309F442
:1003C00041E0842FDF91CF9108958EB588608EBD76
:1003D00089B7806189BF80E197E29BBD8ABD8EB5F8
:1003E00082608EBD089510921B0210921C02109222
:1003F0009D0210929E0210BC83E389B988E98AB9F4
:1004000086E880BD08951F920F920FB60F921124B7
:100410008F939F93EF93FF9380919D02E82FF0E0DD
:100420003196EF77F07080919E0290E0E817F9071F
:1004300031F0E0939D028CB1E35EFD4F8083FF912C
:10044000EF919F918F910F900FBE0F901F90189575
:1004500090919D0280919E029817D1F3E0919E02A7
:10046000F0E03196EF77F070E0939E02E35EFD4F8F
:10047000808108951F920F920FB60F9211248F93CF
:100480009F93EF93FF9390911B0280911C0298170A
:1004900069F0E0911C02F0E03196EF77F070E093A4
:1004A0001C02E556FE4F80818CB901C05598FF9122
:1004B000EF919F918F910F900FBE0F901F90189505
:1004C000482F80911B02282F30E02F5F3F4F2F775E
:1004D000307080911C0290E028173907D1F3F901A0
:1004E000E556FE4F408320931B02559A0895AC01B8
:1004F00017C080911B02282F30E02F5F3F4F2F77CE
:10050000307080911C0290E028173907D1F34F5FBB
:100510005F4FF901E556FE4F608320931B02559A09
:10052000FA016491662329F7089580E690E09F938D
:100530008F93AFD50F900F9008950F931F93CF9384
:10054000DF9347E452E017C080911B02282F30E070
:100550002F5F3F4F2F77307080911C0290E028175B
:100560003907D1F34F5F5F4FF901E556FE4F6083C6
:1005700020931B02559AFA016491662329F7C0E083
:10058000D0E005E610E0DE01AA0FBB1FFD01ED582B
:10059000FE4F60817181FD01ED59FE4F4081518117
:1005A000FD01ED5AFE4F20813181AD5BBE4F8D9133
:1005B0009C917F936F935F934F933F932F939F9360
:1005C0008F93DF93CF931F930F9363D521968DB7AE
:1005D0009EB70C960FB6F8949EBF0FBE8DBFC83065
:1005E000D10589F6DF91CF911F910F9108951F9248
:1005F0000F920FB60F9211243F924F925F926F921B
:100600007F928F929F92AF92BF92CF92DF92EF92A2
:10061000FF920F931F932F933F934F935F936F938B
:100620007F938F939F93AF93BF93CF93DF93EF937A
:10063000FF93809141019091420101969093420174
:10064000809341018091410190914201843691054E
:1006500009F08FC0A6EE4A2EA0E05A2EF6EF8F2E9C
:10066000F0E09F2EE6ED6E2EE0E07E2EAA24BB2465
:1006700033243394E501CC0FDD1F6BE8E62E61E0F7
:10068000F62EEC0EFD1ED7018D919C911197892BB2
:1006900041F08D919C911197019711969C938E93A7
:1006A00053C053E8C52E51E0D52ECA0CDB1CF60111
:1006B00080818823C1F0FE01ED5AFE4F0081118137
:1006C0009CD4CD58DE4F68817981015010406F5F16
:1006D0007F4F52DA080F191FD70111961C930E9302
:1006E000F601108217C0FE01ED5BFE4F0081118103
:1006F00084D4CD59DE4F68817981015010406F5FFD
:100700007F4F3ADA080F191FD70111961C930E93E9
:10071000F6013082F501ED57FE4F2081D301ED91B6
:10072000FC918081D4019C91892B80839C91D20182
:10073000ED91FC91222321F08081892B808304C0DC
:1007400080819095982390830894A11CB11CE2E0CD
:10075000F0E04E0E5F1E0894811C911C6E0E7F1EF1
:10076000F8E0AF16B10409F085CF10924201109263
:100770004101CEE1D1E046EEE42E40E0F42EA6EFBA
:10078000B0E040E050E060E070E0FA01E75CFE4F6E
:100790002081FB01E250FF4F0190F081E02D80812C
:1007A0009881892B8083FB01E25FFE4F0190F081ED
:1007B000E02D9081220F30E08881982309F431E008
:1007C000230FFA01E75CFE4F20838081813029F5F9
:1007D000FA01ED57FE4F2081FB01EA52FF4F0190D5
:1007E000F081E02D80819C91892B80839C91F70181
:1007F000C080D180222329F4F6018081892B808357
:1008000005C0F6018081909598239083FA01EE0F40
:10081000FF1FE557FE4F118210824F5F5F4F6E5FE3
:100820007F4F219682E090E0E80EF91E1196483045
:10083000510509F0AACFFF91EF91DF91CF91BF91C0
:10084000AF919F918F917F916F915F914F913F9168
:100850002F911F910F91FF90EF90DF90CF90BF905D
:10086000AF909F908F907F906F905F904F903F9050
:100870000F900FBE0F901F9018950F931F930BE8CA
:1008800011E0980140E150E063E471E080E090E025
:10089000E6D3980140E150E063E571E080E190E04B
:1008A000DED3980140E150E063E671E080E290E041
:1008B000D6D3980140E150E063E771E080E390E037
:1008C000CED31F910F9108950F931F9303E811E06A
:1008D000980140E150E060E070E083E491E0A5D34E
:1008E000980140E150E060E170E083E591E09DD344
:1008F000980140E150E060E270E083E691E095D33A
:10090000980140E150E060E370E083E791E08DD32F
:100910001F910F9108952F923F924F925F926F9285
:100920007F928F929F92AF92BF92CF92DF92EF927F
:10093000FF920F931F93DF93CF93CDB7DEB7C955C7
:10094000D0400FB6F894DEBF0FBECDBFBDDF8EB571
:1009500088608EBD89B7806189BF80E197E29BBDC9
:100960008ABD8EB582608EBD10921B0210921C0251
:1009700010929D0210929E0210BC83E389B988E90F
:100980008AB986E880BD86E291E09093A2028093C6
:10099000A1029093A00280939F02789440E052E0DD
:1009A00017C080911B02282F30E02F5F3F4F2F7719
:1009B000307080911C0290E028173907D1F34F5F07
:1009C0005F4FF901E556FE4F608320931B02559A55
:1009D000FA016491662329F7B0DD58E0752E4AE0EC
:1009E000C42ED12CCC0EDD1E8E010E5C1F4F30E6C6
:1009F000E32E30E0F32E80913801882309F09AC16C
:100A000047ED50E017C080911B02282F30E02F5F88
:100A10003F4F2F77307080911C0290E028173907E4
:100A2000D1F34F5F5F4FF901E556FE4F608320938E
:100A30001B02559AFA016491662329F720E2622E7F
:100A40005E010894A11CB11C91E1892E912C8C0EA1
:100A50009D1E86E0282E312C2C0E3D1EB2E04B2E22
:100A6000512C4C0E5D1E2CE930E03F932F9311D397
:100A700050E00F900F9090919D0280919E029817E8
:100A8000D1F3E0919E02F0E03196EF77F070E093C1
:100A90009E02E35EFD4F40814D30C1F4F601E50F4B
:100AA000F11D10821F930F9381EA90E09F938F9323
:100AB000DF92CF9200D3ADB7BEB716960FB6F894BB
:100AC000BEBF0FBEADBF019771F675C0483019F0BB
:100AD0004F3709F043C0552371F280911B02282F34
:100AE00030E02F5F3F4F2F77307080911C0290E0F5
:100AF00028173907D1F3F901E556FE4F708220938C
:100B00001B02559A80911B02282F30E02F5F3F4F28
:100B10002F77307080911C0290E028173907D1F3AD
:100B2000F901E556FE4F608220931B02559A809191
:100B30001B02282F30E02F5F3F4F2F7730708091BE
:100B40001C0290E028173907D1F3F901E556FE4F52
:100B5000708220931B02559A51508DCF942F905242
:100B60009F3508F088CF403219F4552309F483CF1C
:100B7000563208F080CF842F81568A3108F4492FED
:100B800080911B02282F30E02F5F3F4F2F7730706E
:100B900080911C0290E028173907D1F3F901E5563E
:100BA000FE4F408320931B02559AF601E50FF11D7D
:100BB00040835F5F60CF8AA9833209F454CF8823D2
:100BC00009F451CF64EA70E0C80126D2009759F4C5
:100BD0008BEA90E09F938F935CD281E08093380101
:100BE0000F900F90A7C06EEA70E0C80115D2009771
:100BF00039F4E3EBF0E0FF93EF934BD29EDC1DC0A2
:100C000068EB70E0C80108D2009709F08AC0BF9273
:100C1000AF922FEB30E03F932F939F928F924BD266
:100C2000ADB7BEB716960FB6F894BEBF0FBEADBF38
:100C3000019731F0FF92EF922CD20F900F9013CFCB
:100C4000E981E930B8F7F0E0EE0FFF1FED5BFE4FF2
:100C5000808191819B838A83E981F0E0EE0FFF1F01
:100C6000DF01AD5ABE4F8D919C919D838C83DF0136
:100C7000AD59BE4F8D919C919F838E83ED58FE4F51
:100C80008081918199878887E8E0F0E0EC0FFD1F73
:100C9000FF93EF933F922F9224E030E02C0F3D1F03
:100CA0003F932F935F924F92BF92AF9284EC90E06C
:100CB0009F938F939F928F92FED1ADB7BEB71E9632
:100CC0000FB6F894BEBF0FBEADBF02970CF4B2CF03
:100CD000E981F0E08A819B81EE0FFF1FDF01AD5BB0
:100CE000BE4F11969C938E938C819D81DF01AD5AEE
:100CF000BE4F11969C938E938E819F81DF01AD59DB
:100D0000BE4F11969C938E9388859985DF01AD58CF
:100D1000BE4F11969C938E93E557FE4F1182108221
:100D2000A2CE61ED70E0C80177D1009709F082CFC3
:100D3000A4DD99CE80913801813009F05CCE46E285
:100D400050E017C080911B02282F30E02F5F3F4FEB
:100D50002F77307080911C0290E028173907D1F36B
:100D60004F5F5F4FF901E556FE4F608320931B02F2
:100D7000559AFA016491662329F75FE3B52EAA24F8
:100D8000A39490919D0280919E029817D1F3E091D7
:100D90009E02F0E03196EF77F070E0939E02E35E02
:100DA000FD4F5081252F2154283000F5E52FF0E02C
:100DB000EE5BFE4FA08230E0D901AA0FBB1FFD0100
:100DC000EA52FF4F60817181FB0180812A503F4FC1
:100DD000F9019081892BFB018083AA51BF4FED91CE
:100DE000FC918081D9019C91892B24C0852F81564B
:100DF000883010F5E52FF0E0EE5DFE4F108290E0B8
:100E0000DC01AA0FBB1FFD01EA52FF4F6081718117
:100E1000FB0120818A509F4FFC013081232BFB0175
:100E20002083AA51BF4FED91FC912081DC018C9170
:100E30008095822380836CC0A52FA053A830A0F595
:100E4000652F70E060537040FB01ED57FE4F40810D
:100E5000B0E09D01220F331FF901EA52FF4F0190CC
:100E6000F081E02D8081AA50BF4F9C91892B808317
:100E7000AC91F901EA51FF4F442339F40190F0811C
:100E8000E02D80818A2B808307C00190F081E02DC6
:100E90008081A095A823A083660F771F65577E4F9A
:100EA000FB011182108234C05B3151F48BEA90E077
:100EB0009F938F93EED0109238010F900F909BCD9F
:100EC00080911B02282F30E02F5F3F4F2F7730702B
:100ED00080911C0290E028173907D1F3F901E556FB
:100EE000FE4F708220931B02559A80911B02282F7F
:100EF00030E02F5F3F4F2F77307080911C0290E0E1
:100F000028173907D1F3F901E556FE4FB08227C003
:100F100080911B02282F30E02F5F3F4F2F773070DA
:100F200080911C0290E028173907D1F3F901E556AA
:100F3000FE4F708220931B02559A80911B02282F2E
:100F400030E02F5F3F4F2F77307080911C0290E090
:100F500028173907D1F3F901E556FE4F5083209346
:100F60001B02559A0ECFA0E0B0E0E8EBF7E065C6B3
:100F7000EC01A880B980CA80DB80A114B104C1044F
:100F8000D10441F484E2A82E89EDB82E8BE5C82E59
:100F900087E0D82EC601B5012DE133EF41E050E0E6
:100FA00029D627EA31E440E050E005D67B018C01E8
:100FB000C601B5012DE133EF41E050E01BD6CA0177
:100FC000B9012CEE34EF4FEF5FEFF5D56E0D7F1DBD
:100FD000801F911F97FF04C061507040804090486F
:100FE000688379838A839B839B013F77C901CDB74F
:100FF000DEB7EAE03EC6B7DF089584E391E0B3DFF1
:101000000895A0E0B0E08093340190933501A0935F
:101010003601B09337010895FB01DC018D910190F9
:1010200080190110D9F3990B0895A0E0B0E0EAE12E
:10103000F8E005C67C01EB018A01690109C0CE0117
:101040002196F6010995F70181937F010150104027
:1010500001151105A1F7CDB7DEB7E8E00CC6A0E099
:10106000B0E0E4E3F8E0EBC5EC017B018A01690143
:1010700009C0F70161917F01CE012196F601099522
:101080000150104001151105A1F7CDB7DEB7E8E01A
:10109000F2C5A0E0B0E0EEE4F8E0D7C5FE01359679
:1010A00061917191AF018091A1029091A20219D03A
:1010B0002096E2E0E6C5AEE0B0E0E0E6F8E0C5C5C7
:1010C00085E08C838B899C899A838983CE0147969E
:1010D000AC016D897E89CE01019646D32E96E2E061
:1010E000D0C5ABE0B0E0E6E7F8E09FC53C012B01DE
:1010F0005A01FC0117821682838181FD03C06FEFC4
:101100007FEFBBC19AE0892E1E010894211C311C7F
:10111000F3012381F20123FD859123FF81912F01AA
:10112000882309F4A7C1853239F423FD859123FF73
:1011300081912F01853221F4B30190E079D4E8CF79
:10114000982FDD24CC249924FFE1FD15D0F09B32AB
:1011500069F09C3228F4903259F0933291F40EC029
:101160009D3249F0903369F441E024C052E0D52A21
:1011700084E0D82A28C098E0D92A25C0E0E1DE2AF8
:1011800022C0D7FC29C0892F80538A3070F4D6FE44
:1011900005C0989C902C1124980E15C0C89CC02C9A
:1011A0001124C80EF0E2DF2A0EC09E3229F4D6FCCC
:1011B00061C140E4D42A07C09C3619F450E8D52A0E
:1011C00002C0983649F4F20123FD959123FF9191D5
:1011D0002F01992309F0B8CF892F8554833018F057
:1011E0008052833038F444E050E0A40EB51E5FE333
:1011F00059830FC0933631F0933779F0933509F066
:1012000052C01FC0F5018081898342E050E0A40EE6
:10121000B51E710101E010E011C0F501E080F18020
:10122000D6FC03C06FEF7FEF02C0692D70E042E093
:1012300050E0A40EB51EC701AED38C015FE7D522E6
:1012400013C0F501E080F180D6FC03C06FEF7FEFA3
:1012500002C0692D70E042E050E0A40EB51EC70147
:101260008FD38C0150E8D52AD3FE06C018C0B30135
:1012700080E290E0DDD3CA948C2D90E00817190726
:10128000B0F30DC0F701D7FC8591D7FE81917F01A6
:10129000B30190E0CDD3C110CA94015010400115A4
:1012A000110581F7E4C0943611F0993669F5D7FE3F
:1012B00008C0F501E080F1800281138144E050E034
:1012C0000AC0F501808191817C010027F7FC00951F
:1012D000102F42E050E0A40EB51E5FE6D52217FFA6
:1012E0000AC010950095F094E094E11CF11C011DDA
:1012F000111D80E8D82A2AE030E0A101C801B70119
:10130000DDD3F82EF2183FC0953729F41D2D1F7E2E
:101310002AE030E01DC01D2D197F9F3661F0903707
:1013200020F4983509F0A6C00FC0903739F09837EF
:1013300009F0A0C004C028E030E00AC0106114FD2C
:10134000146020E130E004C014FD166020E132E0BA
:1013500017FF08C0F501608171818281938144E0AB
:1013600050E008C0F50180819181BC0180E090E0EF
:1013700042E050E0A40EB51EA101A0D3F82EF21851
:101380008FE7D82ED122D6FE0BC05EEFD522F914FE
:1013900038F4D4FE07C0D2FC05C08FEED82202C0BC
:1013A0001F2D01C0192DD4FE0DC0FE01EF0DF11D42
:1013B0008081803319F499EED92208C01F5FD2FED4
:1013C00005C003C08D2D867809F01F5F0D2DD3FC5D
:1013D00013C0D0FE0EC01C1510F09F2C0AC09F2C0D
:1013E0009C0C911A1C2D05C0B30180E290E020D323
:1013F0001F5F1C15C8F304C01C1510F4C11A01C0EE
:10140000CC2404FF0FC0B30180E390E011D302FFAE
:101410001CC001FD03C088E790E002C088E590E0B1
:10142000B3010CC0802F867881F001FF02C08BE2EF
:1014300001C080E2D7FC8DE2B30190E0F9D205C093
:10144000B30180E390E0F4D29A94F914C8F3FA94CB
:10145000F101EF0DF11DB301808190E0E9D2FF2091
:10146000B1F705C0B30180E290E0E2D2CA94CC208B
:10147000C9F74ECEF30166817781CB012B96E2E16D
:10148000F0C3FC0120FD08C023FD05C022FF02C0FF
:1014900073836283518340830895EF92FF920F9389
:1014A0001F9344FF02C033E011C046FF02C034E086
:1014B0000DC0DB01FC01AA0FBB1FEE1FFF1F109424
:1014C000D1F76A0F7B1F8E1F9F1F31E0660F771FBA
:1014D000881F991F3150D1F77B018C01E20EF11C5E
:1014E000011D111DA8019701B701CA011F910F919C
:1014F000FF90EF9008950F931F93CF93DF938C018C
:10150000C80154D2EC0197FD06C04AD3892BC1F71C
:10151000B801CE01B9D2CE01DF91CF911F910F91C9
:101520000895A0E0B0E0E6E9FAE087C3EC01C62E3A
:101530005A01122F3BD2AC018B3219F08D3249F493
:101540001068CA9409F466C0CE0130D2AC0197FD90
:1015500061C06DEFD62ED1228D2D8073F1F4403312
:10156000E1F4CA9409F442C0CE0120D2AC0197FD47
:101570003DC082E0D82A483711F0483551F480E464
:10158000D82ACA9499F1CE0111D2AC0199232CF436
:101590002DC0D6FC02C080E1D82AEE24FF248701AA
:1015A000242F2053283080F0D4FC09C02A3060F06A
:1015B000D6FE05C02F7D822F8151863020F0BE01DE
:1015C000CA0162D210C027504D2DC801B70165DF96
:1015D0007B018C0182E0D82ACA9459F0CE01E6D171
:1015E000AC0197FFDDCFD1FC04C014C0EE24FF2472
:1015F0008701D7FE08C010950095F094E094E11C97
:10160000F11C011D111D2D2DB801A701C50139DFE8
:1016100081E001C080E0CDB7DEB7EAE02AC3A0E2F6
:10162000B0E0E4E1FBE005C36C01A62E8A0179017C
:10163000FE01319680E2DF011D928A95E9F770E0A4
:1016400030E060E040E050E04F01A1E0B0E0F601A2
:101650008381F70183FD259183FF21917F0122235F
:1016600009F47CC02E3519F44115510569F1872F15
:1016700090E08417950744F42D3551F12D3221F473
:10168000332329F431E021C0332309F4622F322FB0
:10169000832F869586958695F401E80FF11D832F9B
:1016A00087703D0102C0660C771C8A95E2F72081A5
:1016B00026292083361711F430E007C0361710F4BE
:1016C0003F5FE6CF3150E4CF71E04F5F5F4FBFCF58
:1016D000332319F08E8180628E83772359F0FE01C7
:1016E00031969E012F5D3F4F808180958193E21757
:1016F000F307D1F7BB24B3944E010894811C911CCD
:10170000C60154D1AC0197FD21C08695869586957A
:10171000F401E80FF11D808190E09A01277030708C
:1017200002C0959587952A95E2F780FD04C0B60121
:10173000CA01AAD10BC00115110519F0D8014D93AA
:101740008D01AA94BB24AA20D9F602C0BB2031F493
:101750000115110529F0F801108202C0EE24FF24C2
:10176000C701A096EEE081C2A0E0B0E0E9EBFBE0AB
:1017700060C25C016B013A01FC0117821682882469
:10178000DCC0812F90E00CD2892B19F0C501B3DEAB
:10179000D4C0153249F4F601F3FC6591F3FE619172
:1017A0006F01653259F415E2C50100D197FDD1C032
:1017B000181709F4C2C0B50167D1D0C06A3219F058
:1017C000162F00E006C0F3FC1591F3FE11916F0196
:1017D00001E099240EC00260692D70E080E090E085
:1017E00040E25BDE962EF601F3FC1591F3FE1191BB
:1017F0006F01212F20532A3070F301FD03C099247B
:101800009A9403C0992009F4A9C0183621F01C3617
:1018100099F4F6010BC0F601F3FC6591F3FE6191BA
:10182000683619F06F01162F07C008600460F3FCDA
:101830001591F3FE11916F01112309F48FC0612FEF
:1018400070E082EC92E091D0892B09F487C0802F60
:1018500000FF03C0EE24FF2407C0F301E080F18005
:1018600022E030E0620E731E1E3649F4F501468117
:10187000578160E070E0202FC70103DE5EC01336A1
:1018800089F481FD02C099249394C5018FD097FDFE
:1018900060C0E114F10419F0F70181937F019A947B
:1018A000A1F749C01B3551F49601A701692DC50167
:1018B000B6DE6C01009709F03EC038C0C5011BDEE2
:1018C00097FD47C01F3641F1103728F4143611F147
:1018D000193621F524C0133719F01537F9F41AC059
:1018E000C50164D0EC0197FD0FC05AD1892B21F0BE
:1018F000B501CE01C9D008C0E114F10419F0F70117
:10190000C1937F019A9461F7E114F104A1F0F7010A
:10191000108211C0006203C0006101C00064202F6A
:10192000A701692DC501FDDD882329F4F501838117
:10193000807379F413C000FF8394F501F380F601FE
:10194000F3FC1591F3FE11916F01112309F019CFEA
:1019500005C0882019F42FEF3FEF02C0282D30E09A
:10196000C901CDB7DEB7EEE080C1FC0105900616D7
:1019700021F00020D9F7C00108953197CF010895D3
:10198000FC010590615070400110D8F7809590954A
:101990008E0F9F1F0895FC0161507040019001104F
:1019A000D8F7809590958E0F9F1F0895CF93DF9362
:1019B000EC014B8140FF1AC046FF0AC04F7B4B83AE
:1019C0008E819F8101969F838E838A81282F2BC0D1
:1019D00042FF13C0E881F9818081282F332727FD3A
:1019E00030952115310529F440624B832FEF3FEFED
:1019F0001BC03196F983E88311C0EA85FB85CE01CF
:101A000009959C0197FF0AC09B812F5F3F4F11F002
:101A100080E201C080E1892B8B83E8CF8E819F819A
:101A200001969F838E8330E0C901DF91CF910895A5
:101A30000F931F93CF93DF938C01EB018B8181FF79
:101A40001BC082FF0DC02E813F818C819D81281794
:101A5000390764F4E881F9810193F983E88306C0CA
:101A6000E885F985802F0995892B31F48E819F8136
:101A700001969F838E8302C00FEF1FEFC801DF9195
:101A8000CF911F910F9108959C01FB01838180FFED
:101A900011C086FD0FC09FEF2F3F390759F02283F9
:101AA00080648F7D83838681978101979783868366
:101AB00030E002C02FEF3FEFC9010895FA01AA27D5
:101AC000283051F1203181F1E8946F936E7F6E5F81
:101AD0007F4F8F4F9F4FAF4FB1E03ED0B4E03CD02F
:101AE000670F781F891F9A1FA11D680F791F8A1F12
:101AF000911DA11D6A0F711D811D911DA11D20D079
:101B000009F468943F912AE0269F11243019305D32
:101B10003193DEF6CF010895462F4770405D419323
:101B2000B3E00FD0C9F7F6CF462F4F70405D4A3370
:101B300018F0495D31FD4052419302D0A9F7EACF38
:101B4000B4E0A6959795879577956795BA95C9F767
:101B500000976105710508959B01AC010A2E06945A
:101B60005795479537952795BA95C9F7620F731F13
:101B7000841F951FA01D0895AA1BBB1B51E107C020
:101B8000AA1FBB1FA617B70710F0A61BB70B881F0D
:101B9000991F5A95A9F780959095BC01CD0108959C
:101BA000911106C0803219F089508550D0F7089500
:101BB000992788270895629FD001739FF001829F23
:101BC000E00DF11D649FE00DF11D929FF00D839FCC
:101BD000F00D749FF00D659FF00D9927729FB00D69
:101BE000E11DF91F639FB00DE11DF91FBD01CF017C
:101BF0001124089597FB092E05260ED057FD04D019
:101C00004BD00AD0001C38F4509540953095219562
:101C10003F4F4F4F5F4F0895F6F790958095709521
:101C200061957F4F8F4F9F4F08952F923F924F9214
:101C30005F926F927F928F929F92AF92BF92CF925C
:101C4000DF92EF92FF920F931F93CF93DF93CDB765
:101C5000DEB7CA1BDB0B0FB6F894DEBF0FBECDBFDD
:101C600009942A88398848885F846E847D848C84AE
:101C70009B84AA84B984C884DF80EE80FD800C81B7
:101C80001B81AA81B981CE0FD11D0FB6F894DEBF9A
:101C90000FBECDBFED010895A1E21A2EAA1BBB1BFA
:101CA000FD010DC0AA1FBB1FEE1FFF1FA217B30728
:101CB000E407F50720F0A21BB30BE40BF50B661F3E
:101CC000771F881F991F1A9469F760957095809502
:101CD00090959B01AC01BD01CF010895F894FFCF11
:101CE0000A0D3F3F00434F4E464947202020202009
:101CF000202020202025752020202020202535751B
:101D000020202020202535752020202020253575F5
:101D10002020202020202535750A0D000A0D3E20A8
:101D2000002573004D414E55414C000A0D004C49B1
:101D30005354000A0D0A0D00434F4E4649470025F3
:101D4000686875002568687525752575257525757C
:101D50000053415645003700370031003100310053
:101D600031003100310038003800320032003200DA
:101D70003200320032000201804020100804350099
:101D800035003500350035003500380038003300A7
:101D900033003300330033003300360036002010A8
:101DA000080402012004000000030000000060029B
:081DB000280200000100000000
:00000001FF
